:1000000080C098C097C096C095C094C093C092C05D
:1000100091C090C08FC08EC08DC08CC08BC08AC074
:1000200089C088C087C062C027090061A08601001E
:1000300062400D030061F049020062F04902006174
:10004000400D030062A086010061E093040062504D
:10005000C3000061C027090074A086010061E0931D
:10006000040074400D030061E093040074E0930405
:100070000061F049020074C027090061F0490200E4
:10008000621027000061F049020074C02709006473
:100090001027000074A0860100641027000074A0DF
:1000A000860100641027000074E093040061F049A9
:1000B0000200621027000061F049020074E093041E
:1000C0000061F0490200621027000061400D03004A
:1000D0006250C3000061400D030062F049020061FC
:1000E000F049020062400D030061A08601006290A9
:1000F000D003006150C3000062C027090030000037
:10010000000011241FBECFEDCDBF10E0A0E6B0E08F
:10011000E0E5F4E003C0C89531960D92A036B10732
:10012000D1F710E0A0E6B0E001C01D92A036B10703
:10013000E1F726C165CF611571058105910581F053
:1001400027E530E040E050E0809A215030404040C8
:10015000504057FFF9CF6150704080409040EBCF46
:1001600008952F923F924F925F926F927F928F925B
:100170009F92AF92BF92CF92DF92EF92FF920F9336
:100180001F93CF93DF93CDB7DEB726970FB6F894C2
:10019000DEBF0FBECDBF69837A838B839C83222E03
:1001A000332E442E552E6E2C7F2C802E912E1E82A7
:1001B0001D82A22EB32EC42ED52EAE0CBF1CC01E87
:1001C000D11E5D2D4C2D3B2D2A2D1AD12115310527
:1001D0004105510549F188B3836088BB952D842D75
:1001E000732D622DA8DF88B38C7F88BB992D882D55
:1001F000772D662DA0DF8D819E8101969E838D8354
:10020000E82EF92E0027F7FC0095102F69817A81DE
:100210008B819C815D2D4C2D3B2D2A2DF1D0E2163A
:10022000F30604071507B8F226960FB6F894DEBF5A
:100230000FBECDBFDF91CF911F910F91FF90EF9037
:10024000DF90CF90BF90AF909F908F907F906F90F6
:100250005F904F903F902F900895EF92FF920F93F1
:100260001F93282F392F220F331F220F331F280FE0
:10027000391FF32FE22FEA5DFF4FC895802D82369C
:10028000D1F485EA95E29BBD8ABDF32FE22FE95DAB
:10029000FF4FC895802D3196C895902D3196C89501
:1002A000A02D3196C895B02D5BE5E52E51E0F52ED9
:1002B000012D112D57C08136F1F482EF95E29BBDDF
:1002C0008ABDF32FE22FE95DFF4FC895802D31964F
:1002D000C895902D3196C895A02D3196C895B02D12
:1002E00042ECE42E41E0F42E012D112D23EC31E0FF
:1002F00040E050E03BC08437D1F48CE696E29BBDF1
:100300008ABDF32FE22FE95DFF4FC895802D31960E
:10031000C895902D3196C895A02D3196C895B02DD1
:1003200033E4E32E33E0F32E012D112D1BC0843670
:1003300011F588EC96E29BBD8ABDF32FE22FE95DB3
:10034000FF4FC895802D3196C895902D3196C89550
:10035000A02D3196C895B02D2DECE22E28E0F22E7E
:10036000012D112D512F402F3F2D2E2D682F792F2C
:100370008A2F9B2FF6DE1F910F91FF90EF9008952B
:10038000CFEDD0E0DEBFCDBF19BE8FEF87BB18BA6F
:1003900082E480BF84E083BF86E286BF80E48FBDB5
:1003A00089E08EBD12BC00E010E0E6E2F0E0C89506
:1003B000802D803371F0CE2FDF2F912F802F4DDFD6
:1003C0000F5F1F4F2596FD2FEC2FC895802D803392
:1003D000A1F783B7887F83BF8EB5887F8EBD85B731
:1003E000806285BF85B7806185BF60E177E280E08C
:1003F00090E0A1DE18BA17BA889580E090E027C097
:10040000A1E21A2EAA1BBB1BEA2FFB2F0DC0AA1FAD
:10041000BB1FEE1FFF1FA217B307E407F50720F06D
:10042000A21BB30BE40BF50B661F771F881F991FE8
:100430001A9469F76095709580959095262F372FBF
:10044000482F592F6A2F7B2F8E2F9F2F0895FFCF74
:00000001FF
